:020000040800F2
:1000000000090020250500081D1A0008ED19000848
:10001000091A0008ED190008011A00082705000850
:10002000270500082705000827050008993500085E
:10003000270500082705000827050008AD3A000835
:1000400027050008270500082705000827050008E0
:100050002705000827050008DD37000809380008D3
:1000600035380008613800088D3800082705000879
:1000700027050008270500082705000827050008B0
:100080002705000827050008270500083D2A000865
:10009000A92A0008FD2A0008512B0008B9380008D9
:1000A0002705000827050008270500082705000880
:1000B0002705000827050008270500082705000870
:1000C0002705000827050008270500082705000860
:1000D0002705000827050008270500082705000850
:1000E0002139000827050008270500082705000812
:1000F0002705000827050008270500082705000830
:10010000270500082705000827050008270500081F
:10011000270500082705000827050008270500080F
:1001200027050008270500082705000827050008FF
:1001300027050008270500082705000827050008EF
:1001400027050008270500082705000827050008DF
:1001500027050008270500082705000827050008CF
:100160004FF0FF0C1CEAD0521EBF1CEAD15392EA9A
:100170000C0F93EA0C0F6FD01A4480EA010C400276
:1001800018BF5FEA41211ED04FF0006343EA5010D0
:1001900043EA5111A0FB01310CF00040B1F5000F12
:1001A0003EBF490041EAD3715B0040EA010062F1C1
:1001B0007F02FD2A1DD8B3F1004F40EBC25008BFAB
:1001C00020F00100704790F0000F0CF0004C08BFC9
:1001D00049024CEA502040EA51207F3AC2BFD2F196
:1001E000FF0340EAC250704740F400004FF00003A4
:1001F000013A5DDC12F1190FDCBF00F000407047DE
:10020000C2F10002410021FA02F1C2F1200200FA1B
:1002100002FC5FEA310040F1000053EA4C0308BFE2
:1002200020EADC70704792F0000F00F0004C02BF33
:10023000400010F4000F013AF9D040EA0C0093F0AE
:10024000000F01F0004C02BF490011F4000F013B08
:10025000F9D041EA0C018FE70CEAD15392EA0C0F76
:1002600018BF93EA0C0F0AD030F0004C18BF31F0E1
:10027000004CD8D180EA010000F00040704790F0B7
:10028000000F17BF90F0004F084691F0000F91F05B
:10029000004F14D092EA0C0F01D142020FD193EA21
:1002A0000C0F03D14B0218BF084608D180EA0100A9
:1002B00000F0004040F0FE4040F40000704740F085
:1002C000FE4040F44000704780F0004002E000BF74
:1002D00081F0004142001FBF5FEA410392EA030F31
:1002E0007FEA226C7FEA236C6AD04FEA1262D2EB7B
:1002F0001363C1BFD218414048404140B8BF5B4280
:10030000192B88BF704710F0004F40F4000020F018
:100310007F4018BF404211F0004F41F4000121F02E
:100320007F4118BF494292EA030F3FD0A2F1010278
:1003300041FA03FC10EB0C00C3F1200301FA03F1B6
:1003400000F0004302D5494260EB4000B0F5000FD9
:1003500013D3B0F1807F06D340084FEA310102F198
:100360000102FE2A51D2B1F1004F40EBC25008BF4A
:1003700020F0010040EA03007047490040EB000014
:10038000013A28BFB0F5000FEDD2B0FA80FCACF115
:10039000080CB2EB0C0200FA0CF0AABF00EBC25042
:1003A00052421843BCBFD0401843704792F0000F30
:1003B00081F4000106BF80F400000132013BB5E783
:1003C0004FEA41037FEA226C18BF7FEA236C21D0F9
:1003D00092EA030F04D092F0000F08BF084670475E
:1003E00090EA010F1CBF0020704712F07F4F04D12C
:1003F000400028BF40F00040704712F100723CBF3F
:1004000000F50000704700F0004343F0FE4040F468
:10041000000070477FEA226216BF08467FEA236326
:100420000146420206BF5FEA412390EA010F40F411
:10043000800070474FF0000304E000BF10F000435D
:1004400048BF40425FEA000C08BF704743F0964344
:1004500001464FF000001CE050EA010208BF70475F
:100460004FF000030AE000BF50EA010208BF7047E6
:1004700011F0004302D5404261EB41015FEA010CFB
:1004800002BF84460146002043F0B64308BFA3F1F3
:100490008053A3F50003BCFA8CF2083AA3EBC253D5
:1004A00010DB01FA02FC634400FA02FCC2F12002F4
:1004B000BCF1004F20FA02F243EB020008BF20F02B
:1004C0000100704702F1200201FA02FCC2F1200291
:1004D00050EA4C0021FA02F243EB020008BF20EA86
:1004E000DC70704742000ED2B2F1FE4F0BD34FF0DA
:1004F0009E03B3EB126209D44FEA002343F000439A
:1005000023FA02F070474FF00000704712F1610FBC
:1005100001D1420202D14FF0FF3070474FF000008E
:10052000704700BF02E000F000F8FEE772B6264810
:1005300080F30888254880F3098825482549086004
:10054000022080F31488BFF36F8F03F075F803F077
:10055000D9F84FF0553020491B4A91423CBF41F831
:10056000040BFAE71D49194A91423CBF41F8040BBC
:10057000FAE71B491B4A1C4B9A423EBF51F8040B39
:1005800042F8040BF8E700201849194A91423CBF91
:1005900041F8040BFAE703F053F803F0B5F8154CF3
:1005A000154DAC4203DA54F8041B8847F9E700F014
:1005B0003FF8124C124DAC4203DA54F8041B884742
:1005C000F9E703F03BB8000000090020001100200B
:1005D0000000000808ED00E00001002000090020F4
:1005E000B83B000800110020241100202811002031
:1005F000D4250020600100086001000860010008A7
:10060000600100082DE9F04FC1F80CD0C3689D4689
:10061000BDE8F08F002383F311882846A04700200F
:1006200002F036FDFEE702F0CFFC00DFFEE700003F
:10063000F8B500F03BFE02F04DFF074602F098FFD0
:10064000064600283ED12B4B9F423BD001339F42B0
:100650003BD0294B27F0FF029A4239D1F8B200F083
:10066000FFFB354642F2107400F000FC08B1002494
:10067000254601F041F978B30024032000F042F848
:10068000254636B11D4B9F4203D0002402F068FF7F
:100690002546002002F028FF194B9B6813F0400309
:1006A0001FD00DB100F044F800F042FC01F0B8F9A1
:1006B0000546C4B101F0B4F9401BA04213D900F0C3
:1006C00037F8F3E735460024CEE704460125CBE7AB
:1006D00005464FF47A74C7E7B4F57A7F08BF012561
:1006E000CFE71C46E0E700F0D5FC012002F0D6FC85
:1006F000DFE700BF010007B0000008B0263A09B0EC
:10070000000C0140084B187003280CD8DFE800F0FB
:1007100008050208022000F025BE022000F01ABEE3
:100720000022024B5A607047281100202C11002033
:1007300038B501F0E1F830B103221F4B1A700022E6
:100740001E4B5A6038BD1E4B1E4A19680131F9D044
:1007500004339342F9D11C4C194DD4F80424AA4215
:10076000F0D31A4B9B6803F1006303F5C8439A4228
:10077000E8D202F0C9FE02F0DBFE002000F0B0FD7E
:100780000220FFF7BFFF124BDA690022DA61D96954
:1007900099699A619B6972B64FF0E023C3F8085DCE
:1007A0003021D4F80034D4F8042481F311889D4614
:1007B00083F308881047C5E7281100202C1100207A
:1007C0000064000820640008006000080011002098
:1007D0000010024049F26900084A136899B21B0CE4
:1007E00000FB013344F250611360054B186882B27C
:1007F000000C01FB0200186080B27047201100203D
:100800001C11002010B504460021102200F0C6FD86
:10081000034B03CB206061601868A06010BD00BF6F
:10082000E8F7FF1FF0B5ADF5517D6EAC4FF4C47223
:1008300007460D462046002100F0B0FD01F0F0F81B
:100840004FF47A72B0FBF2F0244B186093E8070083
:10085000022384E807000DF5ED702382FFF7D2FF35
:100860004EF603031E4907A8238403F057F91E23FD
:100870000DF2EB2284F832310DF1340C07AB1E4639
:1008800003CE664510605160334602F10802F6D18E
:1008900030681060B3880FAE314693802046012245
:1008A00000F0C8FD00230393AB7E80B2029305F1F4
:1008B000190301930123CDE904600093384605A391
:1008C000D3E90023E97E01F0FFFB0DF5517DF0BD7A
:1008D000AFF300809E6AC421818A46EE3411002065
:1008E0002C3B00082DE9F041264D80462B7A0C4622
:1008F000DAB0FBB9204627A900F0C2FE074600285F
:1009000036D19DF89D60C82E32D801464FF4FA7258
:10091000284600F043FD32460DF19E0105F1090025
:1009200000F02AFD9DF89C302E4477722B720BB993
:10093000E37E2B728122002106AD27A800F02EFD58
:100940000122294627A800F0E1FE00230393A37E9D
:1009500080B2029304F1190301932823CDE90450D6
:100960000093404605A3D3E90023E17E01F0ACFBF0
:100970005AB0BDE8F08100BFAFF30080264172722B
:10098000DF25D7B77C210020F0B54FF48A7500240D
:10099000234EF1B005FB006596F8D830D8222146E9
:1009A00085F8DC3085F8E8403AA800F0F7FC06F15D
:1009B000090000F0EBFCD5F8E430C2B206AF8DF8C8
:1009C000F00006F109010DF1F100CDE93A3400F033
:1009D000D3FC394601223AA800F0CEFE80B2CDE920
:1009E000047008230127CDE9023706F1D8030193EB
:1009F0003023317A00930B4807A3D3E9002301F099
:100A000063FBA04206DD01F00BF8C5F8E0003846B4
:100A100071B0F0BD2046FBE778F6339F93CACD8DC9
:100A20007C2100204C210020F0B51E4E1E4F1F4D92
:100A300085B0304601F074FB044660B310220021FB
:100A4000684600F0ABFC4FF00003227B6068A168B1
:100A500062F303038DF8003002AB03C3019B2268ED
:100A6000384662F31C0301939DF800306A4643F058
:100A700020038DF800300023194602F0E1F9044606
:100A800020B9304601F050FB2C70D2E72B78072BB1
:100A900003D801332B7005B0F0BD024801F044FBD0
:100AA000F9E700BF4C210020A82300207523002077
:100AB00070B50D4614461E4601F062FA50B9022E7A
:100AC00010D1012C0ED112A3D3E900230120C5E9D6
:100AD000002307E0282C10D005D8012C09D0052CC4
:100AE0000FD0002070BD302CFBD10BA3D3E9002325
:100AF000ECE70BA3D3E90023E8E70BA3D3E900233A
:100B0000E4E70BA3D3E90023E0E700BFAFF30080E5
:100B1000401DA12026812A0B78F6339F93CACD8DE4
:100B20009E6AC421818A46EE26417272DF25D7B7BC
:100B3000F017304A39059E5638B505460E4C00214F
:100B4000013500F0EFFBA4F8F051B4F8F00100F02B
:100B5000D1FB78B1B4F8F00100F0DCFB014648B9F4
:100B6000B4F8F00100F0DEFBB4F8F0310133A4F882
:100B7000F031EAE738BD00BF7C2100202DE9F04FBD
:100B80008DB000AF04460D4601F0FAF9002848D1B7
:100B90002B7E022B1AD1EB8A012B17D100F040FFDC
:100BA0000646FFF717FE4FF4C873B0FBF3F202FBE3
:100BB0001303DFF88C829BB206F516763344C8F82F
:100BC0000030EB7E33B900229E4B1A703437BD469D
:100BD000BDE8F08F284607F11C0100F005FD002854
:100BE000F4D107F10C00FFF70DFEBD7F07F10C01FA
:100BF0002A4607F11F0002F061FF0028E3D10F2D04
:100C000008D8904B1D70D8F80030A3F51673C8F8BB
:100C10000030DBE7397F0029D8D0204601F0A8F961
:100C2000D4E7EB8A282B6BD010D8012B63D0052B8F
:100C3000CCD1BFF34F8F8449844BCA6802F4E06281
:100C40001343CB60BFF34F8F00BFFDE7302BBDD107
:100C50007F4CEA7E237A9A42B8D194F8DC206B7EEE
:100C60009A4240F0E480284604F1EA0100F0B8FD21
:100C700006460028AAD1012384F8E83000F0D0FE0F
:100C8000D4F8E030C01A192840F6B83338BF19201C
:100C9000984228BF1846FFF7CDFB6E49FFF760FA70
:100CA00005462068FFF7C6FB6B49FFF759FA014676
:100CB0002846FFF70FFBFFF715FC20604FF48A7200
:100CC00094F8D930606802FB03F562197B6092F8F2
:100CD000E83053B1D2F8E430E946834215D000231E
:100CE00082F8E830C2F8E030CD4663685B4A9B0A80
:100CF000013313816AE729462046FFF793FD65E734
:100D000029462046FFF7EEFD60E7B2F8EC803B6035
:100D100008F1030A4FEA9A0A4FEA8A02D11DC9086C
:100D2000A9EBC1039D46EB460021584600F036FB77
:100D300005F1EE0142465846214400F01DFB3B6898
:100D400013B9012000F0CCFA94F8D20000F0D2FAE6
:100D5000054630B9207200F0EDFA284600F0C0FADE
:100D6000C2E7D4F8D4303BB994F8D200B4F8F031EB
:100D7000834201D8FFF7E0FED4F8D43043449D42CB
:100D800008D294F8D200B4F8F0310130834201D88F
:100D9000FFF7D2FE594660685FFA8AF200F006FB60
:100DA00008B9CD468AE7636894F8D200434463608B
:100DB000D4F8D43008EB030AC4F8D4A000F09AFAAF
:100DC000824509D394F8D230D4F8D4000133401BC3
:100DD00084F8D230C4F8D400B8F1FF0F0FD8002542
:100DE000257200F0A7FA284600F07AFA00F084FD98
:100DF0001A4B188108B9FFF79BFCCD46E6E64FF485
:100E00008A727B6894F8D90002FB0343D3F8E4208C
:100E100083F8E86002F58072C3F8E060C3F8E4206C
:100E2000FFF7B2FDFFF700FE84F8D960B9E740F69E
:100E3000B8322368FA33934294BF23602260C5E638
:100E4000482100204521002000ED00E00400FA05C3
:100E50007C210020CDCCCC3D6666663F341100205D
:100E6000014B1870704700BF4011002030B54FF0A3
:100E70000054264B226885B09A4217D1637DABB1EE
:100E80000025234A23481370237DC9220372224977
:100E9000C0F8E450093000F06FFA2046E0222946FD
:100EA00000F07CFA0124204605B030BD02F06AFB58
:100EB000044608B90024F6E7184A194DD36943F0EF
:100EC0000073D361AA6D174B9A42F3D12B6E013B8D
:100ED0007E2BEFD8144A01AB07CA83E807001846F7
:100EE000032100F0D9FC6B6D83424FF00003E1D188
:100EF0002A6D8A4203BFAB652A6E054B1C4601BFB3
:100F00001A70EA6D094B1A60CDE700BF9AAD44C56F
:100F1000401100207C21002016000020001002401B
:100F2000006600405041A0B05866004018110020F3
:100F30002DE9F04385B000F0DFFC0223494C6371DA
:100F400000230293484B2081D3F800C0BCF57A7F80
:100F500012D3464F464BB7FBFCF59C458CBF0A238A
:100F60001123B5FBF3F603FB1652591EC8B2002A33
:100F70003ED002290B46F4D89DF80B303D495A1E4D
:100F80009DF80A303C48013B1B0443EA0253BDF87C
:100F90000820013A13434B6001F042FF0023019304
:100FA000364B374900934FF48052364B364800F0A9
:100FB000B5FF364B197811B1334800F0D9FF00F076
:100FC0002FFD0546FFF706FC4FF4C873B0FBF3F2A4
:100FD00002FB130305F516709BB218442C4B1860E6
:100FE00002F0C6FA08B10F23238105B0BDE8F083F3
:100FF000731EB3F5806FBFD24FF47A75C0EBC00E8D
:101000000EF103034FEAE30909FB0555C3F3C703D8
:10101000C11AC9B209F101088844B5FBF8F5B5F564
:10102000617F08D90EF1FF33C3F3C703C11A581EFD
:101030000F28C9B214D84A1E072A8CBF00220122E9
:10104000581800FB0660B7FBF0F7BC4594D1002AA6
:1010500092D0ADF808608DF80A308DF80B108BE750
:101060001346EDE73411002018110020005125022D
:101070003F420F0010110020A8230020B10A0008F1
:10108000441100207D0B00084C210020401100205D
:10109000482100202DE9F04F80A7D7E900670FF223
:1010A0000429D9E90089734D93B00DF1300AFFF797
:1010B000BBFC18220021504600F070F9DFF8B8B1EF
:1010C0006E4C002352461946584601F0E1FE014697
:1010D00050BB102208A800F061F9E36883F0100308
:1010E000E36000F09FFC0DF1240C0B4612A90246B0
:1010F00011E903008CE803009DF83410C1F30300EC
:10110000890649BF0E99BDF83810C1F31C0141F0A2
:10111000004158BFC1F30A018DF82C000891284600
:1011200008A901F0E1F9CCE7284600F029FF0446C0
:10113000002847D100F074FCDFF844B1DBF8003040
:1011400098423FD300F06CFC0790FFF743FB4FF44D
:10115000C873B0FBF3F101FB1300079A83B202F5E9
:1011600016701844CBF80000DFF818B18DF8204055
:101170009BF8001011B901238DF8203050460791DB
:10118000FFF740FB07990DF12100C1F11004E4B213
:10119000062C28BF06245144224600F0EDF808AB87
:1011A000039318230293384B013401930123E4B2D3
:1011B000009332463B462846049400F027FF002364
:1011C0008BF8003000F02CFC304A314C1368C31A05
:1011D000B3F57A7F30D3106000F024FC02460B4652
:1011E000284600F0ABFF284600F0CAFE20B3237A61
:1011F000DFF8A0B0002B14BF032302238BF80530C7
:1012000000F00EFC4FF47A73B0FBF3F00122CBF840
:1012100000005146584600F0BFF9182302931E4BB8
:1012200080B2019340F25513CDE903A000934246EA
:101230004B46284600F0EAFE237ABBB100F0F0FBF3
:1012400094F8E83073B9D4F8E03043B1C01A236899
:10125000FA2B38BFFA230533B0EB430F02D300203B
:10126000FFF792FB237A002B7FF41FAF13B0BDE88A
:10127000F08F00BF4C210020A8230020000801406F
:101280004821002045210020442100207023002017
:101290007C2100203411002074230020401DA12057
:1012A00026812A0BF1C6A7C1D068080F70B501F0DE
:1012B000CDFF0024084E094D3080286833888342D2
:1012C00008D901F0BFFF2B6804440133B4F5C84FBF
:1012D0002B60F2D370BD00BFA42300207823002030
:1012E00002F042B800F10060920000F5C84001F041
:1012F000E7BF0000054B1A68054B1B889B1A834209
:1013000002D9104401F09EBF0020704778230020CE
:10131000A4230020024B1B68184401F099BF00BFB2
:1013200078230020024B1B68184401F0A3BF00BFC4
:1013300078230020064991F8243033B10023082295
:10134000086A81F82430FFF7CDBF0120704700BF45
:101350007C230020022802BF1022014B1A61704733
:1013600000080140022802BF4FF48012014B1A61AD
:10137000704700BF00080140002310B5934203D01E
:10138000CC5CC4540133F9E710BD000003460246AB
:10139000D01A12F9011B0029FAD170470346024402
:1013A000934202D003F8011BFAE770472DE9F84396
:1013B0001F4D144695F824200746884652BBDFF897
:1013C00070909CB395F824302BB92022FF21484619
:1013D0002F62FFF7E3FF95F824004146C0F10802B1
:1013E000A24228BF224605EB8000D6B29200FFF74A
:1013F000C3FF95F82430A41B1E44F6B2082E1744F0
:101400009044E4B285F82460DBD1FFF793FF002815
:10141000D7D108E02B6A03EB82038342CFD0FFF7DA
:1014200089FF0028CBD10020BDE8F8830120FBE72D
:101430007C2300202DE9F3470D4604460021904609
:10144000284640F27912FFF7A9FF23462022002107
:10145000284600F0EBFF022220212846231D00F041
:10146000E5FF032222212846631D00F0DFFF03224F
:1014700025212846A31D00F0D9FF10222821284647
:1014800004F1080300F0D2FF08223821284604F1B5
:10149000100300F0CBFF08224021284604F111037D
:1014A00000F0C4FF08224821284604F1120300F08E
:1014B000BDFF20225021284604F1140300F0B6FF9E
:1014C00040227021284604F1180300F0AFFF0822E3
:1014D000B021284604F1200300F0A8FF0822B8211B
:1014E000284604F1210300F0A1FFC02604F12207E1
:1014F0003B46314608222846083600F097FFB6F5ED
:10150000A07F07F10107F3D194F8323031468DF80E
:101510000730082228460DF1070300F087FF002658
:1015200004F1330A9DF807304FEAC6099E4209F5D7
:10153000A47720D394F83231502B28BF50238DF854
:101540000730B8F1000F08D13946072228460DF1BF
:10155000070300F06BFF09F24F17002604F2331463
:101560009DF8073007EBC6019E420DD30731C8082E
:1015700002B0BDE8F0870AEB060308223946284688
:1015800000F054FF0136CDE7A3190822284600F0E9
:101590004DFF0136E4E7000038B50C460021054652
:1015A00021600346C4F803102046202200F03EFFCD
:1015B00020462B1D0222202100F038FF20466B1D03
:1015C0000322222100F032FF2046AB1D03222521F9
:1015D00000F02CFF20461022282105F1080300F01E
:1015E00025FF072038BD0000F7B5047F05460E46ED
:1015F0002CB1838A122B02D9012003B0F0BD002345
:10160000072219462846009600F0D2FD731C00936D
:10161000012200230721284600F0CAFDD4B9B31CDB
:101620000093052223460821284600F0C1FD0D2421
:10163000B378102BE0D83746B278BB1B934210D357
:101640002B7F0734A88AE408B3B9844294BF0020F2
:101650000120D2E7AB8A0824DB00083BDB08B3702B
:10166000E6E7FB1C2146009308220023284600F0F1
:101670009FFD08340137DFE7201A18BF0120BCE7BF
:10168000F7B5047F05460E462CB1838ACA2B02D9D2
:10169000012003B0F0BD0023082219462846009619
:1016A00000F086FD731CD4B908220093114623462E
:1016B000284600F07DFD10247378C82BE8D801235C
:1016C00072785F1C013B934210D32B7F0734A88AAA
:1016D000E408B3B9844294BF00200120D9E7AB8A63
:1016E0000824DB00083BDB087370E5E7F3192146AB
:1016F000009308220023284600F05AFD08343B4698
:10170000DEE7201A18BF0120C3E70000F7B50D4639
:1017100004460021164628468122FFF73FFE234655
:1017200008220021284600F081FE94F90120637808
:10173000002AB8BF7F238DF807309EB90722082101
:1017400028460DF1070300F071FE0F270026023432
:101750009DF8073007EBC6019E4205D30731C80844
:1017600003B0F0BD0827F1E7A3190822284600F0CE
:101770005DFE0136ECE70000F7B50E460546002198
:1017800014463046CE22FFF709FE2B4628220021C0
:10179000304600F04BFE2B7AC82B28BFC8238DF8AB
:1017A00007308CB90822282130460DF1070300F0DC
:1017B0003DFE30242F469DF807207B1B934205D326
:1017C000E01DC00803B0F0BD2824F3E7214607F16F
:1017D00009030822304600F029FE08340137EAE701
:1017E000F7B5047F05460E4634B1838AB3F5827F90
:1017F00002D9012003B0F0BD0123102200212846A8
:10180000009600F0D5FCDCB9B31C009309222346F6
:101810001021284600F0CCFC19247388B3F5807F92
:10182000E7D837467288BB1B934210D32B7F07340F
:10183000A88AE408B3B9844294BF00200120D9E704
:10184000AB8A1024DB00103BDB087380E5E73B1D0F
:101850002146009308220023284600F0A9FC083402
:101860000137DFE7201A18BF0120C3E730B5094D63
:101870000A4491420DD011F8013B5840082340F32F
:101880000004013B2C4013F0FF0384EA5000F6D122
:10189000EFE730BD2083B8ED4FF0FF33F7B500EB35
:1018A00081061946DFF848C0DFF848E0B0421BD097
:1018B00050F8042B01AF0192042217F8014B81EA82
:1018C000046108240D46DB184941013C002DBCBFD2
:1018D00083EA0C0381EA0E0114F0FF04F2D1013A0D
:1018E00012F0FF02E9D1E1E7D843C94303B0F0BDEC
:1018F0009336EAA9EBE1F042F7B56B46354A10683A
:1019000051686A4603C308233349344802F0E6F8B5
:10191000044690BB0A256B46314A106851686A46F6
:1019200003C308232F492D4802F0D8F804460028A5
:1019300047D00369B3F5CE3F43D8B0F86620B2F57F
:101940007A7F3ED1284A024402F15C018B4238D3AF
:101950005C3B224900209E1AFFF788FF074632466B
:10196000002004F16401FFF781FFA3689F4228D1A2
:10197000E368984208BF002523E00369B3F5CE3F32
:1019800026D8428BB2F57A7F20D1174A024402F161
:1019900010018B4218D3103B104900209D1AFFF70D
:1019A00065FF06462A46002004F11801FFF75EFF96
:1019B000A3689E4202D1E368984201D00D25AAE7B0
:1019C0000025284603B0F0BD1025A4E70C25A2E7AA
:1019D0000B25A0E74C3B0008DC9B010000640008DD
:1019E000553B0008909B0100089CFFF7EFF309832B
:1019F000EFF30583014B9B6BFEE700BF00ED00E0BA
:101A000008B5FFF7F3FF0000EFF30983EFF3058359
:101A1000014B5B6BFEE700BF00ED00E0FEE700005E
:101A200001F008BD01F0B4BC2DE9F041456A15B9DB
:101A30004162BDE8F0814B68AC4623F06047C3F3D8
:101A40008A4616EA230638BF3E464FEAD37EC3F3E2
:101A500080782B465A68BEEBD27F22F060440AD0D1
:101A6000002A18DAA40CB44217D19D420FD10D60A0
:101A7000DEE71346EEE7A74207D102F08044C2F347
:101A8000807242450BD054B1EFE708D2EDE7CCF8B5
:101A900000100B60CDE7B44201D0B442E5D81A681B
:101AA0009C46002AE5D11960C3E700002DE9F04704
:101AB0004FF47F49089D01F007044FEAD5082244FE
:101AC00005F0070500EBD100944201D1BDE8F08795
:101AD00004F0070705F0070A57453E4638BF56464B
:101AE000111BC6F108068E4228BF0E46E108415C74
:101AF00008EBD50E13F80EC0B94029FA06F721FA03
:101B00000AF1FFB28CEA010147FA0AF739408CEA80
:101B1000010C03F80EC034443544D5E7082341F2E4
:101B2000210280EA012001B24000002980B203F1C5
:101B3000FF33B8BF504013F0FF03F4D170470000EB
:101B400038B50C468D18A54200D138BD14F8011BDC
:101B5000FFF7E4FFF7E700000346406848B102687A
:101B600099895A605A89013292B291425A8138BF9A
:101B70009A81704770B504460D4688B02022002136
:101B80006846FFF70BFC20460495FFF7E5FF024689
:101B900058B16B46054608AE1C4603CCB4422860DB
:101BA0006960234605F10805F6D1104608B070BDFE
:101BB000082817D909280CD00A280CD00B280CD0DB
:101BC0000C280CD00D280CD00E2814BF402030203B
:101BD00070470C2070471020704714207047182061
:101BE0007047202070470000082817D90C280CD90E
:101BF00010280CD914280CD918280CD920280CD955
:101C000030288CBF0F200E207047092070470A2013
:101C100070470B2070470C2070470D207047000064
:101C20002DE9F843078C0446072F1ED9D0E9029806
:101C300000254FF6FF73C5F12006A5F1200029FA13
:101C400005F108FA06F628FA00F031430143C9B25B
:101C50001846FFF763FF0835402D0346EBD13A469F
:101C6000E169BDE8F843FFF76BBF4FF6FF70BDE8D1
:101C7000F883000010B54B6823B9CA8A63F30902E0
:101C8000CA8210BD04691A681C600361C38A013BE3
:101C9000C3824A60EFE700002DE9F84F1D46CB8A6A
:101CA0000F46C3F309010529814692460B4630D001
:101CB0000020AAB207F11A049EB2042E1FFA80F87F
:101CC0000FD8904503F1010306D3FB8A0A4462F35F
:101CD00009030120FB821AE01AF800600130E65483
:101CE000EAE79045F1D21C23A1F1050BBBFBF3F20F
:101CF00003FB12BB7C681FFA8BF6002C45D14846CB
:101D0000FFF72AFF044638B978606FF00200BDE89B
:101D1000F88F4FF00008E6E70026066078604FF085
:101D2000000BADB2454510D90AEB0803221D13F88C
:101D3000011B08F101089155B1B21B291FFA88F85F
:101D40002BD0454506F10106F1D8FB8AC3F3090201
:101D5000154465F30903BCE71C46013292B22368BF
:101D6000002BF9D16B1F0B441C21B3FBF1F30133A2
:101D70009BB29A42D3D2BBF1000FD0D14846FFF7B5
:101D8000EBFE20B9C4F800B0BFE70122E7E7C0F8D6
:101D900000B05E4620600446C1E74545D5D94846B7
:101DA000FFF7DAFE08B92060AFE7C0F800B0002600
:101DB00020600446B6E700002DE9F74F1C465B693A
:101DC000074688460092002B00F0A480238C2BB19C
:101DD000E269002A00F09E80072B33D807F10C003F
:101DE000FFF7BAFE054628B96FF00205284603B092
:101DF000BDE8F08F14220021FFF7D0FA228CE169B0
:101E000005F10800FFF7B8FA208C48F000410130D6
:101E100080B2FFF7E9FEFFF7CBFE013880B22084E5
:101E2000013028746369228C1B782A4403F01F0355
:101E300063F03F031372384669602946FFF7F4FDEB
:101E40000125D3E7072202339BB20633B3FBF2F33B
:101E5000C18A828A9BB2521A92B29342C4D84FF07E
:101E600000094FF0800A4E464D4600F10C030193E5
:101E70000198FFF771FE83460028B5D01422002197
:101E8000FFF78CFA002E3BD10222009BABF8083002
:101E90000BF1080E1FFA82FC0CF10100BCF1060FD9
:101EA000218C80B201D88E422CD3FFF79DFEFFF724
:101EB0007FFE8E4208BF4FF0400A626901381278F7
:101EC00080B202F01F0242EA49120BEB00014AEA1B
:101ED000020A013048F0004281F808A08BF8100097
:101EE00059463846CBF80420FFF79EFD238C013578
:101EF000B3424FF0000A2DB289F00109B8D175E75D
:101F00000022C5E7E169895D01360EF80210B6B21C
:101F10000132BFE76FF0010568E70000F8B504463D
:101F200015460E46302200211F46FFF737FA069B62
:101F3000B5F5001F6360079B28BF4FF6FF72A362D1
:101F40004FF0000338BF6A09A760E66197B204F159
:101F500010009A4206D800230360A782E3822383FD
:101F6000E360F8BD0660013330462036F1E700003B
:101F700003781BB94BB2002BC8BF0170704700003B
:101F800000787047F8B50C46C969074611B9238C2B
:101F9000002B37D1257E1F2D34D8387828BB228CD2
:101FA000072A2CD8268A36F003032BD14FF6FF7070
:101FB000FFF7C6FD4FF6FF7220F001003602400425
:101FC00046EA0565400C45EA402523462946384641
:101FD000FFF7F2FE002807DD626913780133DBB2F8
:101FE0001F2B88BF00231370F8BD218A2D0645EAF8
:101FF000012505432046FFF713FE0246E5E76FF093
:102000000300F1E76FF00100EEE7000070B5044651
:102010001D4616468AB0282200216846FFF7BEF901
:10202000BDF838306946ADF810300F9B2046059357
:102030009DF84030CDE902658DF81830119B07936B
:10204000BDF84830ADF82030FFF79CFF0AB070BDF6
:102050002DE9F041D36905460C4616460BB9138CA1
:102060005BBB377E1F2F28D895F80080B8F1000F92
:1020700026D03046FFF7D4FD3378210241EAC33140
:1020800041EA0801338A41EA076141EA0341024615
:102090003346284641F08001FFF78EFE00280ADD16
:1020A0003378012B07D1726913780133DBB21F2B10
:1020B00088BF00231370BDE8F0816FF00100FAE7DC
:1020C0006FF00300F7E70000F0B504460D461E462A
:1020D00017468BB0282200216846FFF75FF99DF86C
:1020E0004C3029465A1E534253418DF800309DF81A
:1020F00040306A46ADF81030119B204605939DF89C
:102100004830CDE902768DF81830149B0793BDF85E
:102110005430ADF82030FFF79BFF0BB0F0BD00004E
:10212000406A00B104307047436A1A68426202692B
:102130001A600361C38A013BC38270472DE9F041F5
:10214000D0F8208014461D4641460027174E09B995
:10215000BDE8F081D1E90223A21A65EB03039642A0
:1021600077EB03031ED2036A8B420DD1FFF782FD8A
:10217000036A1B68036203690B60C38A0161016A19
:10218000013B8846C382E2E7FFF774FD0B68C8F89D
:10219000003003690B60C38A0161013BC382D8F838
:1021A0000010D4E788460968D1E700BF80841E008C
:1021B0002DE9F04F8BB00D4614469B468046DDF866
:1021C0005090002800F01A81B9F1000F00F016813C
:1021D000531E3F2B00F21281012A03D1BBF1000FE5
:1021E00040F00C810023CDE90833B8F81430B5EB8A
:1021F000C30F4FEAC30703D300200BB0BDE8F08F35
:102200002B199F42D8F80C3036BF7F1B2746FFB2F0
:102210001BB9D8F81030002B7BD0272D4ED8C5F134
:102220002806B7424FF0000334BF3E46F6B2009393
:1022300029463246D8F8080008ABFFF737FCA7EB71
:10224000060A35445FFA8AFA2821B8F8143003F1F7
:102250000053053BDB000493D8F80C300393039B39
:1022600013B1BAF1000F2CD1D8F8100040B1BAF177
:10227000000F05D05246009608AB691AFFF716FC0E
:1022800038B2002FB8D066070AD00AAB03EBD401EE
:1022900011F8083C624202F00702134101F8083CC1
:1022A000082C3DD9102C40F2B680202C40F2B8808A
:1022B000BBF1000F00F09D80082335E0BA460026F0
:1022C000C2E7049BE02B28BFE02306930B44AB42FC
:1022D000059315D95A1B924538BF5246039828BF1B
:1022E000D2B20096691A08AB04300792FFF7DEFB02
:1022F000079A1644AAEB020A1544F6B25FFA8AFA64
:10230000049B069A05999B1A0493039B1B680393ED
:10231000A5E700933A462946D8F8080008ABADE790
:10232000BBF1000F13D00123B4EBC30F6CD0082C0A
:1023300012D89DF82030621E23FA02F2D50706D586
:102340004FF0FF3202FA04F423438DF820309DF859
:10235000203089F8003050E7102C12D8BDF820301A
:10236000621E23FA02F2D10706D54FF0FF3202FABD
:1023700004F42343ADF82030BDF82030A9F8003034
:102380003BE7202C0FD80899631E21FA03F3DA07E4
:1023900005D54FF0FF3202FA04F40C430894089B71
:1023A000C9F8003029E7402C2BD0DDE90865611E13
:1023B000C4F12102A4F1210326FA01F105FA02F287
:1023C00025FA03F311431943CB0712D50122A4F1D7
:1023D0002003C4F1200102FA03F322FA01F1A24022
:1023E000524243EA010363EB430332432B43CDE9FB
:1023F0000823DDE90823C9E90023FEE66FF00100A8
:10240000FBE66FF00800F8E6082CA0D9102CB3D931
:10241000202CEED8C3E7BBF1000FADD0022383E739
:10242000BBF1000FBBD004237EE70000012A30B5CA
:10243000144638BF01220025402A28BF402285B01B
:10244000012CCDE9025517D81B788DF808305307B9
:102450000AD004AB03EBD20515F8083C544204F053
:102460000704A34005F8083C0346009102A8002198
:10247000FFF71CFB05B030BD082CE5D9102C03D8A4
:102480001B88ADF80830E2E7202C02D81B680293C5
:10249000DDE7D3E90045CDE90245D8E710B5CB68C3
:1024A0001BB98B600B618B8210BD04691A681C60BC
:1024B0000361C38A013BC382CA60F0E703064CBFD5
:1024C000C0F3C0300220704708B50246FFF7F6FFA0
:1024D000022806D15306C2F30F2001D100F00300F9
:1024E00008BDC2F30740FBE72DE9F04F93B0CDE9FB
:1024F00003230A6804461046FFF7E0FF02280CBFDA
:102500000026C2F30626002A0D46824680F2FD818F
:1025100012F0C04940F0F981097B002900F0F581F3
:10252000022803D02378B34240F0F281C2F304635F
:102530001046069302F07F030593FFF7C5FF059B46
:1025400000224FEA8348002348EA0A48294448EA1F
:102550004668CE78CDE90823F309834648EA0008A7
:10256000029367D0059B0246009320465346676856
:1025700008A9B847002800F0CE81276A4FB9414624
:1025800004F10C00FFF7F6FA074690B96FF002006D
:1025900054E03B6998450DD03F68002FF9D1414682
:1025A00004F10C00FFF7E6FA07460028EED0236A94
:1025B0003B60276297F817C006F01F08CCF3840C25
:1025C000ACEB08001FFA80FE0028B8BF0EF1200017
:1025D000A8EB0C031FFA83FEB8BF00B2002B0793D1
:1025E000BEBF0EF120031BB20793D7E9022152EAC6
:1025F000010338D04FF0000C039BDFF800E29A1A79
:10260000049B63EB010196457CEB01032BD36B7BB1
:1026100097F81AE0734519D1029B002B78D0012856
:1026200021DC7868F8B9DFF8D8C1944570EB010374
:1026300016D337E0276A27B96FF00C0013B0BDE856
:10264000F08F3B699845B5D03F68F4E76C489042FD
:102650007CEB010301D30020F0E7029B002BFAD0B2
:10266000079B0F2B17DCFA7DB30002F0030203F087
:102670007C031343FB7539462046FFF7FBFA6B7B5F
:10268000BB76029B3BB9FB7DC3F38402013262F34C
:102690008603FB75D0E76A7BBB7E9A42DBD1029B47
:1026A000002B35D0B309022B32D0039B1422BB6020
:1026B000049B0021FB600DA8FEF770FE039B2046E3
:1026C0000A93049BADF83EB00B932B1D0C932B7B10
:1026D0008DF840A0013BDBB2ADF83C30069B8DF895
:1026E00041808DF84230059B0AA98DF8433094F85B
:1026F0002C3083F001038DF84430A3689847FB7DAC
:10270000C3F38403013303F01F039B02FB82A2E7A0
:10271000FB7DC6F34012B2EBD31F40F0FF80C3F342
:102720008403434540F0FD80029A2B7BB609002AC2
:1027300052D016F0010665D1032B40F2F580039BC1
:102740003946BB60049B04F10C00FB60FB8A66F316
:102750000903FB822B7BAE1D033B3246DBB2FFF746
:102760009BFA00280CDA39462046FFF783FAFB7DF6
:10277000C3F38403013303F01F039B02FB8205E7CD
:10278000AB88DDE908843B834FF6FF73C9F1200075
:10279000A9F1200228FA09F104FA00F0014324FA11
:1027A00002F211431846C9B2FFF7B8F909F1080956
:1027B000B9F1400F0346E9D13146B8822A7B033A8A
:1027C000D2B2FFF7BDF9FB7DB882DA43C2F3C01283
:1027D00062F3C713FB753EE7A6B92E1D013B3246D7
:1027E0003946DBB204F10C00FFF756FA0028BADBD9
:1027F0002A7B3146013AB88AD2B2E2E780841E00D1
:1028000040420F00F98A013BC1F309010429DAB201
:102810005DD80023281D07F11B069A4208D910F83D
:1028200001CB013306F801C001310529DBB2F4D137
:10283000934228BF0023039938BF04330A910499B7
:1028400038BFDBB20B9107F11B010C91796838BFDF
:102850005B190D910E93FB8AADF83EB0C3F30903EB
:102860001A44069BADF83C208DF84230059B8DF84C
:1028700040A08DF8433094F82C308DF8418083F0DF
:1028800001038DF8443000237B602A7BB88A013A2B
:10289000291DFFF755F93B8BB882834203D12046AF
:1028A000A3680AA9984720460AA9FFF7F7FDFB7D10
:1028B000BA8AC3F38403013303F01F039B02FB8234
:1028C0003B8B9A420CBF00206FF01000B6E67B688D
:1028D000002BADD0052001E033461C301E68002ED1
:1028E000FAD1091A081D2E1D184401EB090CBCF180
:1028F0001B0F5FFA89F39BD89A4299D916F8013BCE
:1029000009F1010900F8013BEFE76FF0090095E6D6
:102910006FF00A0092E66FF00B008FE66FF00D008B
:102920008CE66FF00E0089E66FF00F0086E600BFC0
:10293000F0B53F4D3F4FEB6943F00073EB61EB693E
:102940003D4B9B6AD3F800623E4046F00106C3F857
:102950000062D3F800423C4044EA002444F0010401
:10296000C3F80042002955D000200646C3F81C02D7
:10297000C3F80402C3F80C02C3F8140203EBC0044A
:1029800001300E28C4F84062C4F84462F6D1002732
:102990004FF0010C9678148816F0010F18BFD3F889
:1029A00004E20CFA04F01CBF40EA0E0EC3F804E285
:1029B00016F0020F18BFD3F80CE203EBC4041CBFDF
:1029C00040EA0E0EC3F80CE2760748BFD3F8146253
:1029D00007F1010744BF0643C3F814625668B942C1
:1029E000C4F84062966802F10C02C4F84462D3F85D
:1029F0001C4240EA0400C3F81C02CBD1D3F80022E9
:102A000022F00102C3F80022EB6923F00073EB61AE
:102A1000EB69F0BD0122C3F84012C3F84412C3F8B9
:102A20000412C3F81412C3F80C22C3F81C22E5E701
:102A3000001002400000FFFFA8230020184A08B53C
:102A4000916A8B688B6013F0010104D013F00C0FB6
:102A500018BF4FF48031D80506D513F4406F14BF6A
:102A600041F4003141F00201D80306D513F4402FA0
:102A700014BF41F4802141F00401D3690BB108482F
:102A80009847302383F311880021064800F022FB89
:102A9000002383F31188BDE8084000F0ABBD00BF00
:102AA000A8230020B023002038B5124CA36ADD68AB
:102AB000AA0712D05A6922F002025A61A36913B11F
:102AC000012120469847302383F3118800210A48CA
:102AD00000F000FB002383F31188EB0606D51021DC
:102AE000A36AD960236A0BB102489847BDE8384011
:102AF00000F080BDA8230020B823002038B5124C78
:102B0000A36A1D69AA0712D05A6922F010025A61FD
:102B1000A36913B1022120469847302383F311881B
:102B200000210A4800F0D6FA002383F31188EB064F
:102B300006D51021A36A1961236A0BB10248984790
:102B4000BDE8384000F056BDA8230020B82300207F
:102B500038B50F4CA36A5D682A075D600AD5042268
:102B600022701A6822F002021A60636A13B100210F
:102B7000204698476B0706D5A36A9969236A13B163
:102B8000034809049847BDE8384000F033BD00BF52
:102B9000A823002010B50E4C204600F02FF90D4B55
:102BA0000B211320A36200F009F90B21142000F07F
:102BB00005F90B21152000F001F90B21162000F07A
:102BC000FDF8BDE8104000220E201146FFF7B0BE10
:102BD000A8230020006400400F4B10B59842044623
:102BE00005D10E4BDA6942F00072DA61DB6901222D
:102BF000A36A1A60A36A5A68D20707D56268516847
:102C00001268D9611A60064A5A6110BD0121082074
:102C100000F0B0F9EEE700BFA8230020001002404A
:102C20005B87010003291AD8DFE801F0020A0F14BC
:102C3000836A9B6813F0E05F14BF01200020704797
:102C4000836A9868C0F380607047836A9868C0F3AD
:102C5000C0607047836A9868C0F3007070470020B6
:102C60007047000010B5032927D8DFE801F00227DC
:102C70002B2F836A9968C1F30161183103EB0113AB
:102C80001078840648BF5468C0F3001158BF948878
:102C90004FEA410148BF41EAC40100F00F0058600B
:102CA00048BF41F00401906858BF41EA4451D268DE
:102CB00041F001019860DA60196010BD836A03F584
:102CC000C073DDE7836A03F5C873D9E7836A03F548
:102CD000D073D5E701290AD002290FD081B9836AC0
:102CE000DA68920701D1186903E001207047836A0E
:102CF000D86810F0030018BF01207047836AF2E71C
:102D00000020704710B539B9836AD96889071BD18B
:102D10001B699C0704D110BD012915D00229FAD1E5
:102D2000816AD1F8C031D1F8C441D1F8C80110612D
:102D3000D1F8CC015061202008610869800717D1C3
:102D4000486940F0100012E0816AD1F8B031D1F842
:102D5000B441D1F8B8011061D1F8BC015061202014
:102D6000C860C868800703D1486940F00200486124
:102D7000C3F34000C3F38001000140EA4111107920
:102D800020F030000143117189064BBF9168118911
:102D9000DB085B0D4CBF63F31C0163F30A0113797D
:102DA00048BF916064F3030313714FEA14234FEAA1
:102DB000144458BF118113705480ACE701220901FB
:102DC00000F1604303F56143C9B283F8001300F0DA
:102DD0001F039A4043099B0003F1604303F56143DD
:102DE000C3F880211A607047090100F16040C9B240
:102DF00000F56D4001767047FFF7CCBE01230370EC
:102E0000002300F10802C0E9022200F11002C0E92B
:102E10000422C0E90633C0E908334360704700006C
:102E200010B53023044683F31188022341600370F8
:102E3000FFF7D2FE04230020237080F3118810BD19
:102E40002DE9F0411F4604460D461646302383F314
:102E5000118800F108082378052B0DD0294620465B
:102E6000FFF7E0FE40B1204632462946FFF7FAFE62
:102E7000002080F3118808E03946404600F01AF936
:102E80000028E8D0002383F31188BDE8F08100001A
:102E90002DE9F0411F4604460D461646302383F3C4
:102EA000118800F110082378052B0DD02946204603
:102EB000FFF710FF40B1204632462946FFF722FFB8
:102EC000002080F3118808E03946404600F0F2F80F
:102ED0000028E8D0002383F31188BDE8F0810000CA
:102EE00000238268037503691B6899689142FBD2CD
:102EF0005A6803604260106058607047002382681F
:102F0000037503691B6899689142FBD85A6803608E
:102F1000426010605860704708B50846302383F35C
:102F200011880B7D032B05D0042B0DD02BB983F317
:102F3000118808BD00228B691A604FF0FF3383614E
:102F4000FFF7CEFF0023F2E7D1E9003213605A60A9
:102F5000F3E70000FFF7C4BF054BD9680875186890
:102F6000026853601A6001220275D860FDF74ABBFF
:102F7000D823002030B50C4B0446DD684B1C87B0CD
:102F80000FD02B466846094A00F0CAF82046FFF7E2
:102F9000E3FF009B13B1684600F0CAF8A86907B0C8
:102FA00030BDFFF7D9FFF9E7D8230020192F00081B
:102FB000044B1A68DB6890689B68984294BF0020B5
:102FC00001207047D8230020084B10B51C68D86832
:102FD000226853601A6001222275DC60FFF78EFFC1
:102FE00001462046BDE81040FDF70CBBD823002069
:102FF00038B501230025064C064907482370656053
:1030000000F03EFB0223237085F3118838BD00BF1A
:1030100030250020643B0008D823002000F09AB837
:103020008B60022308618B82084670478368A3F196
:10303000440243F8142C026943F8442C426943F8D3
:10304000402C094A43F8242CC268A3F1200043F81D
:10305000182C022203F80C2C002203F80B2C034A34
:1030600043F8102C704700BF15060008D823002035
:1030700008B5FFF7DBFFBDE80840FFF76BBF0000B6
:10308000024BDB6898610F20FFF766BFD823002052
:10309000302383F31188FFF7F3BF000008B5014622
:1030A000302383F311880820FFF764FF002383F3A4
:1030B000118808BD064BDB6839B1426818605A6058
:1030C000136043600420FFF755BF4FF0FF30704797
:1030D000D823002038B504460D462068844200D12C
:1030E00038BD036823605C608561FFF733FFF4E758
:1030F00010B50A4C23699A6891420CD85A688160CD
:103100000360426010609A685860511A99604FF0ED
:10311000FF33A36110BD1B68891AECE7D823002098
:10312000C0E90323002310B410BC4361FFF7E0BFE4
:10313000036881689A680A449A60426813605A601A
:1031400000234FF0FF320360014B9A61704700BFCC
:10315000D823002070B5124D2A46EB690133EB618C
:1031600052F8103F934206D030269A68013A9A608E
:103170002C69A36803B170BDD4E900210A605160D5
:10318000236083F311882046D4E90331984786F3FE
:10319000118861690029EBD02046FFF7A9FFE7E716
:1031A000D8230020054A30B5D369D2E908451B1B56
:1031B000181945F10001C2E9080130BDD8230020EB
:1031C00000207047FEE70000704700004FF0FF301E
:1031D00070470000BFF34F8F024AD368DB07FCD46F
:1031E000704700BF0020024008B5074B1B7853B959
:1031F000FFF7F0FF054B1A69120641BF044A5A60F7
:1032000002F188325A6008BD4825002000200240A3
:103210002301674508B5054B1B7833B9FFF7DAFF83
:10322000034A136943F08003136108BD4825002059
:10323000002002407F289ABF00F500308002002065
:10324000704700004FF48060704700008020704796
:103250007F2808B50BD8FFF7EDFF00F58063026803
:10326000013204D104308342F9D1012008BD00208D
:10327000FCE700007F2810B504461CD8FFF7AAFF22
:10328000FFF7B2FFF3220D4B4FF48061DA600222A8
:103290001A61FFF7CFFF58611A6942F040021A61C4
:1032A000FFF798FF00F02EF9FFF7B4FF2046BDE8C6
:1032B0001040FFF7CDBF002010BD00BF002002402E
:1032C0002DE9F843054612F00100144606D04FF4EC
:1032D000517200201E4B1A60BDE8F8831D4BAA18DE
:1032E0009A4204D940F24932194B1A60F4E7FFF7C9
:1032F0007BFF4FF00109FFF76DFFDFF85C806D1A6F
:10330000012C0F4605EB010603D8FFF783FF0120D0
:10331000E2E73B88C8F8109033800020FFF75AFF9F
:10332000C8F81000338831F8022B9BB29A420CD0B7
:103330004FF45872064B1A60084B1E60084B1C6015
:10334000084B1F60FFF766FFC6E7023CD8E700BFE7
:1033500044250020000002080020024038250020FB
:10336000402500203C250020084908B50B7828B1ED
:103370001BB9FFF739FF01230B7008BD002BFCD0F0
:10338000BDE808400870FFF745BF00BF4825002092
:1033900038B5EFF31185BDBBEFF30584C4F3080422
:1033A0003023C4B183F31188FFF7FCFE44014B01C5
:1033B000241A43EAD06363EB0103A2009B001218B6
:1033C00043EA947341EB0301C900D00041EA527112
:1033D00085F3118838BD83F31188FFF7E3FE4501BB
:1033E0004B012D1A43EAD06363EB0103AA009B0053
:1033F000121843EA957341EB0301C900D00041EA7A
:10340000527184F3118838BDFFF7CCFE44014B01A3
:10341000241A43EAD06363EB0103A2009B00121855
:1034200043EA947341EB0301C900D00041EA5271B1
:1034300038BD00BF38B5FFF7ABFF00230F4A104C73
:10344000C00840EA4170A0FB025EC908A0FB040C62
:10345000A1FB0440A1FB02121CEB050C5B411CEB21
:10346000040C43EB000011EB0E0142F10002411885
:1034700042F10000090941EA007038BDA59BC42053
:10348000CFF753E310B5094C013AD2B2FF2A00D16D
:1034900010BD500854F82030013054F820009BB281
:1034A00043EA004341F8043BEEE700BF046C0040F0
:1034B00010B50748013AD2B2FF2A00D110BD0C88DE
:1034C000530840F823404C88013340F82340F1E78B
:1034D000046C004007B50122002001A9FFF7D2FFCC
:1034E000019803B05DF804FB13B50446FFF7F2FF43
:1034F000A04205D00122002001A90194FFF7D8FFC6
:1035000002B010BD7047000045F25552064B1A60DC
:1035100003225A6040F2FF729A604CF6CC421A6065
:103520000122024B1A7070470030004050250020E5
:10353000034B1B781BB14AF6AA22024B1A60704754
:103540005025002000300040044B1A682AB902F1CF
:10355000804202F50432526A1A6070474C250020FE
:103560004FF08072014B5A62704700BF001002405A
:1035700008B5FFF7E9FF024B1868C0F3407008BDBB
:103580004C25002008B5FFF7DFFF024B1868C0F399
:10359000007008BD4C250020EFF30983203383F32E
:1035A0000988002383F3118870470000302080F3DE
:1035B000118862B60C4B0D4AD96821F4E061090408
:1035C000090C0A43DA60D3F8FC20094942F0807202
:1035D000C3F8FC200A6842F001020A602022DA7770
:1035E00083F82200704700BF00ED00E00003FA05F9
:1035F000001000E0302310B583F311880B4B5B689B
:1036000013F400630FD0EFF309844FF08073203C74
:10361000E36184F30988FFF7CBFC10B1044BA3618D
:1036200010BD044BFBE783F31188F9E700ED00E0E0
:10363000270600082A06000870470000FEE7000081
:103640000A4B0B480B4A90420BD30B4BC11EDA1CA2
:10365000121A22F003028B4238BF00220021FDF72C
:103660009DBE53F8041B40F8041BECE7DC3B00084C
:10367000D4250020D4250020D4250020FEE700001A
:1036800070B5002504461A4B86B058608562016308
:103690000E46FFF78BFF04F11003C4E904334FF02B
:1036A000FF33A361134BE561D9692B460A462046D7
:1036B000C4E9082304F134018023C4E900440E4A1C
:1036C000A560E5622565FFF7ABFC01230B4AE060CE
:1036D00003750092726868460192B268CDE90223D0
:1036E000074BCDE90435FFF7C3FC06B070BD00BF42
:1036F00030250020D8230020703B0008753B0008CF
:103700007D36000800F030B808B500F063F9FFF727
:103710006FFCBDE80840FFF717BF000070470000CE
:103720004FF0FF310E4B1A6919611A6900221A61B4
:103730001869D868D960D968DA60DA68DA6942F05D
:103740008052DA61DA69DA6942F00062DA61054AC8
:10375000DB69136843F48073136000F01BB900BF8A
:103760000010024000700040194B1A6842F001023C
:103770001A601A689007FCD51A6802F0F9021A60FC
:1037800000225A605A6812F00C0FFBD11A6842F4FA
:1037900080321A601A689103FCD55A6842F4E81224
:1037A0005A601A6842F080721A601A689201FCD559
:1037B0001221084A5A60084A11605A6842F002020F
:1037C0005A605A6802F00C02082AFAD1704700BF0A
:1037D0000010024000641D0000200240084A08B5A5
:1037E000516913680B4003F00103536123B1054A8B
:1037F00013680BB150689847BDE80840FFF7FABE60
:103800000004014054250020084A08B55169136896
:103810000B4003F00203536123B1054A93680BB1D7
:10382000D0689847BDE80840FFF7E4BE00040140B7
:1038300054250020084A08B5516913680B4003F06D
:103840000403536123B1054A13690BB150699847CA
:10385000BDE80840FFF7CEBE00040140542500201B
:10386000084A08B5516913680B4003F00803536117
:1038700023B1054A93690BB1D0699847BDE8084068
:10388000FFF7B8BE0004014054250020084A08B5DF
:10389000516913680B4003F01003536123B1054ACB
:1038A000136A0BB1506A9847BDE80840FFF7A2BE03
:1038B0000004014054250020174B10B55A691C68BC
:1038C000144004F478725A61A30604D5134A936A2B
:1038D0000BB1D06A9847600604D5104A136B0BB140
:1038E000506B9847210604D50C4A936B0BB1D06BF3
:1038F0009847E20504D5094A136C0BB1506C984700
:10390000A30504D5054A936C0BB1D06C9847BDE86C
:103910001040FFF76FBE00BF000401405425002097
:103920001A4B10B55A691C68144004F47C425A6161
:10393000620504D5164A136D0BB1506D98472305E7
:1039400004D5134A936D0BB1D06D9847E00404D5AC
:103950000F4A136E0BB1506E9847A10404D50C4A60
:10396000936E0BB1D06E9847620404D5084A136F6A
:103970000BB1506F9847230404D5054A936F0BB1E0
:10398000D06F9847BDE81040FFF734BE00040140F7
:1039900054250020062108B50846FFF70FFA062136
:1039A0000720FFF70BFA06210820FFF707FA062188
:1039B0000920FFF703FA06210A20FFF7FFF9062185
:1039C0001720FFF7FBF9BDE8084006212820FFF784
:1039D000F5B9000008B5FFF7A3FE054800F00CF8A4
:1039E000FFF70AFAFFF79AFEBDE8084000F002B8B8
:1039F0007C3B000800F042B8002319461C4A013302
:103A0000102BC2E9001102F10802F8D1194B9A6992
:103A100042F07D029A619B690268174BDA60826806
:103A20005A6042681A60C26803F58063DA604269CE
:103A30005A6002691A608269C3F80C24026AC3F8EA
:103A40000424C269C3F80024426AC3F80C28C26A7D
:103A5000C3F80428826AC3F80028026BC3F80C2C50
:103A6000826BC3F8042C426BC3F8002C704700BF74
:103A70005425002000100240000801404FF0E023D0
:103A8000044A08215A6100229A6107220B201A6118
:103A9000FFF7AAB93F19010008B5302383F3118855
:103AA000FFF7BCFA002383F3118808BD08B5FFF7C0
:103AB000F3FFBDE80840FFF79DBD000010B50139D8
:103AC0000244904201D1002005E0037811F8014F33
:103AD000A34201D0181B10BD0130F2E72DE9F041DF
:103AE0009BB10446C91A1778014403F1FF3C8C428C
:103AF000204601D9002008E005780134BD42F6D106
:103B00000CEB0405D618A54201D1BDE8F08115F8EB
:103B1000018D16F801EDF045F5D0E8E7034611F800
:103B2000012B03F8012B002AF9D170476F72672E21
:103B30006172647570696C6F742E663130332D520A
:103B4000616E676546696E646572000040A2E4F1CB
:103B5000646891060041A3E5F265699207000000E0
:103B600063300000603B0008302400203025002036
:103B70006D61696E0069646C6500000000180000EA
:103B800044444144445449440100000042444444F4
:103B900044444444000000004444444444444444F5
:103BA00000000000444444444444444400000000F5
:103BB0004444444444444444E803000000000000FA
:103BC000009C0100000000006400000000000000F4
:0C3BD00040420F00FE2A0100D204000059
:00000001FF
